:103800000C94341C0C944F1C0C944F1C0C944F1CA7
:103810000C944F1C0C944F1C0C944F1C0C944F1C7C
:103820000C944F1C0C944F1C0C944F1C0C944F1C6C
:103830000C944F1C0C944F1C0C944F1C0C944F1C5C
:103840000C944F1C0C944F1C0C944F1C0C944F1C4C
:103850000C944F1C0C944F1C0C944F1C0C944F1C3C
:103860000C944F1C0C944F1C11241FBECFEFD4E0BE
:10387000DEBFCDBF11E0A0E0B1E0ECE1FFE302C0AC
:1038800005900D92A030B107D9F712E0A0E0B1E0A9
:1038900001C01D92A434B107E1F70C94501F0C94A1
:1038A000001C0F92AF93BF93CF93DF93EF93FF93DF
:1038B000FC01EA01DB01C895099231961197D9F70D
:1038C000FF91EF91DF91CF91BF91AF910F9008954C
:1038D0000F921F920F93AF93BF93CF93DF93EF930A
:1038E000FF93FC01EA01DB010990199001E043D04C
:1038F00032961297C9F7FC0103E03DD005E03BD0BA
:10390000FF91EF91DF91CF91BF91AF910F911F90F8
:103910000F9008950F931F93EF93FF93FC0103E023
:103920002AD000E810E0E00FF11FE617F707B9F71B
:10393000FF91EF911F910F9108950F930F9222D055
:10394000082E09E018D00F900F9108950F930F9251
:10395000EF93FF9317D0FC0160935700C895802D1B
:10396000FF91EF910F900F9108950F930BD001E10C
:1039700002D00F910895F999FECF00935700E89572
:10398000FFFF00000091570000FDFCCF089589E083
:103990008093C4008091C10088618093C100089524
:1039A0008091C100877E8093C10008958093C600F6
:1039B0008091C00086FFFCCF8091C000806480931E
:1039C000C00008958091C600992708958091C00095
:1039D0009927807890700895EF92FF920F931F932C
:1039E000CF93DF937B01C0E0D0E0C617D70770F418
:1039F0008C010E94E61C8823E1F30E94E21CF8017E
:103A000081938F012196CE15DF0598F381E090E038
:103A1000DF91CF911F910F91FF90EF900895EF925A
:103A2000FF920F931F93CF93DF937C018B01C0E034
:103A3000D0E0C017D10738F4F70181917F010E94CF
:103A4000D61C2196F6CF81E090E0DF91CF911F91B7
:103A50000F91FF90EF90089540E050E0481759070C
:103A600050F429EC38E000002150304037FFFBCF04
:103A70004F5F5F4FF3CF08950E94D01C0E9400005B
:103A800008950E94E61C8823E1F30E94E21C803224
:103A900019F481E090E0089585E10E94D61C80E051
:103AA00090E0089590E0282F33272138310589F0E0
:103AB0002238310524F42038310549F00DC0223870
:103AC000310549F02839310539F493E005C092E019
:103AD00003C091E001C092E1892F9927089540E049
:103AE00050E0609140017091410146175707D0F4B2
:103AF0002091420230914302E2E4F1E032BD21BD67
:103B00002F5F3F4F808180BDFA9AF99AF999FECFD5
:103B10004F5F5F4F31964617570780F3309343024C
:103B200020934202089540E050E06091400170917E
:103B3000410146175707B0F42091420230914302E9
:103B4000E2E4F1E032BD21BD2F5F3F4FF89A80B52E
:103B500081934F5F5F4F46175707A0F3309343029F
:103B6000209342020895CF93DF93C0E0D0E080918C
:103B7000400190914101C817D907A0F4CE018E5B96
:103B80009E4F2091420230914302220F331FAC011D
:103B900060E870E0C9018C0F9D1F0E94681CC0582E
:103BA000DF4FE5CF0E94B51CDF91CF910895809142
:103BB00042029091430242E451E0609140017091D1
:103BC0004101880F991F0E94511C0895CF93C0E0B6
:103BD00069E081E090E00E94A61C992784FF03C061
:103BE0008F7E0E949D1C0E94E61C8823E1F30E94A8
:103BF000E21C9927823591051CF5803591050CF062
:103C00005CC08134910509F462C0823491057CF472
:103C100081339105B1F18233910524F4C09709F401
:103C20004CC038C18034910509F438C133C18234A5
:103C3000910509F45FC08534910509F45EC02AC17D
:103C40008635910509F4F1C0873591054CF482352C
:103C5000910509F45FC08535910509F469C01AC161
:103C60008437910509F4A4C0853791052CF4843676
:103C7000910509F476C00EC18537910509F4C5C0D8
:103C800009C10E94411D882309F4ADCF84E10E943F
:103C9000D61C81E40E94D61C86E50E94D61C82E5D3
:103CA0000E94D61C80E20E94D61C83E50E94D61C8E
:103CB00084E50E94D61C8BE406C00E94411D882327
:103CC00009F491CF84E10E94D61C80E1E4C061E058
:103CD00070E080E091E00E94EC1C0E94411D88236E
:103CE00009F481CF84E10E94D61C809100010E94DA
:103CF000521DE9CF64E170E008C061E070E080E04F
:103D000091E00E94EC1C64E070E080E091E00E9491
:103D1000EC1CD3CF0E94411D882309F464CF60E0DE
:103D200070E480E090E00E948A1C0E94B51CCACF1B
:103D300062E070E080E091E00E94EC1C0E94411D76
:103D4000882309F450CF2091000180910101992727
:103D5000982F8827820F911D9093430280934202EF
:103D6000B1CF63E070E080E091E00E94EC1C209114
:103D70000101809100019927982F8827820F911DBA
:103D80009093410180934001BC0182E491E00E9444
:103D9000EC1C0E94411D882309F425CF809102016B
:103DA000863419F40E94B31D8DCF0E946F1D8ACFF7
:103DB00063E070E080E091E00E94EC1C2091010142
:103DC000809100019927982F8827820F911D909349
:103DD0004101809340010E94411D882309F403CFD3
:103DE00080910201863419F40E94D71D02C00E94FE
:103DF000931D84E10E94D61C6091400170914101A5
:103E000082E491E00E940F1D60CF0E94411D882333
:103E100009F4E9CE84E10E94D61C8EE10E94D61CF2
:103E200084E90E94D61C86E04ECF64E070E080E01A
:103E300091E00E94EC1C0E94411D882309F4D3CE1E
:103E400084E10E94D61C80910001803531F480917C
:103E50000101882361F4C82F17C0883531F480919F
:103E60000101883061F4C3E00FC0803531F48091E6
:103E70000101883049F4C2E007C0883529F48091F7
:103E80000101882309F4C1E069E08C2F99270E9481
:103E9000A61C19CF85E10E94D61CA5CECF9108950E
:103EA000CFEFD4E0DEBFCDBFCEE1F894AEEFB1E00E
:103EB0000E94851F802D843B79F4AFEFB1E00E9412
:103EC000851F802D833C41F4ADEFB1E00E94851F3A
:103ED000802D9927809366000E94C71C0E94E21CD7
:103EE00084E690E00E942C1D0E94E61C882319F0B5
:103EF0000E94E61D04C0C150C5B9CC2389F70E94B9
:103F00003C1D80E090E00C948D1FF999FECFB2BD6E
:0C3F1000A1BDF89A119600B40895FFCFEF
:0400000300003800C1
:00000001FF
